:020000040800F2
:100000000040002049410008550800085708000832
:1000100000000000000000000000000000000000E0
:100020000000000000000000000000005908000867
:1000300000000000000000005B0800085D080008E8
:100040009941000899410008994100089941000828
:100050009941000899410008994100089941000818
:100060009941000865080008994100089941000875
:1000700099410008994100089941000899410008F8
:1000800099410008994100089941000899410008E8
:1000900099410008994100089941000899410008D8
:1000A00099410008994100089941000899410008C8
:1000B0009941000899410008994100087508000815
:1000C0000448054B10B5834203D0044B002B00D0ED
:1000D000984710BD88010020880100200000000022
:1000E00006480749091A8910CB0F591810B549104D
:1000F00003D0044B002B00D0984710BD880100208E
:10010000880100200000000010B5074C2378002B68
:1001100009D1FFF7D5FF054B002B02D0044800E0C2
:1001200000BF0123237010BD8801002000000000E3
:100130009C410008054B10B5002B03D0044905482D
:1001400000E000BFFFF7CCFF10BDC046000000007C
:100150008C0100209C41000870B50D4E0D4DAD1B6B
:10016000AD1006D00024A300F35801349847A542EF
:10017000F9D104F013F8084E084DAD1BAD1006D0B0
:100180000024A300F35801349847A542F9D170BD6B
:1001900010430008104300081043000814430008EF
:1001A00010B5034B0100186800F0B2F810BDC0464E
:1001B0000000002010B5034B0100186800F052F851
:1001C00010BDC04600000020F0B5830746D0541E85
:1001D000002A42D0CEB20200032502E01A00013C00
:1001E0003BD3531C16702B42F8D1032C2DD9FF2280
:1001F0000A40150215432A0415430F2C16D927006F
:10020000103F3F093E01B4461E001A0010366644F6
:10021000156055609560D5601032B242F8D10F225A
:1002200001373F01DB191440032C0ED9261FB608F5
:10023000B700BC461A001F1D674420C2BA42FCD159
:1002400003220136B6009B191440002C05D0C9B218
:100250001C19197001339C42FBD1F0BD140003003E
:10026000C3E7C04670B50500002915D00C1F2368F0
:10027000002B27DB280000F0C3F8244B1A68002A63
:1002800005D0A2420CD92168601882421CD062605D
:1002900028001C6000F0B6F870BDA34203D81A0015
:1002A0005368002BF9D111685018A04219D012D808
:1002B00021686018834221D063605460280000F0F8
:1002C000A1F8E9E7E418D5E710685268844661446C
:1002D00021606260DCE70C2328002B6000F092F8BC
:1002E000DAE720680918501811608342E6D11868CF
:1002F0005B688446614411605360DFE718685B689F
:1003000084466144216063605460D7E7A401002003
:10031000F8B50323CD1C9D43083506000C2D2AD2C9
:100320000C25A94229D8300000F06AF82A4F3A6813
:10033000002A0AD013685B1B04D440E023685B1BCF
:100340001FD522005468002CF8D17B68002B3DD0CB
:100350002900300000F042F8431C29D00323C41CBC
:100360009C43A04205D0211A300000F037F8431C0E
:100370001ED025600AE0002DD3DA0C230020336064
:10038000F8BD0B2B0FD92360E4182560300000F076
:1003900039F8200007220B30231D9043C31AEFD0F9
:1003A0005A42E250ECE7A2420DD063685360EDE799
:1003B0000C233000336000F025F80020E0E7140043
:1003C0000B2BE0D854683C601400DFE700213000BC
:1003D00000F004F87860BBE7A4010020002370B5AA
:1003E000064C05000800236000F00EF8431C00D006
:1003F00070BD2368002BFBD02B60F9E7B40A002006
:100400007047C0467047C046044A1368002B00D1AD
:10041000034B1818106018007047C046AC0100204C
:10042000B80A0020002243088B4274D303098B4290
:100430005FD3030A8B4244D3030B8B4228D3030CB4
:100440008B420DD3FF22090212BA030C8B4202D356
:100450001212090265D0030B8B4219D300E0090A7E
:10046000C30B8B4201D3CB03C01A5241830B8B4287
:1004700001D38B03C01A5241430B8B4201D34B0370
:10048000C01A5241030B8B4201D30B03C01A5241D5
:10049000C30A8B4201D3CB02C01A5241830A8B425A
:1004A00001D38B02C01A5241430A8B4201D34B0243
:1004B000C01A5241030A8B4201D30B02C01A5241A7
:1004C000CDD2C3098B4201D3CB01C01A524183095B
:1004D0008B4201D38B01C01A524143098B4201D395
:1004E0004B01C01A524103098B4201D30B01C01AC0
:1004F0005241C3088B4201D3CB00C01A524183083A
:100500008B4201D38B00C01A524143088B4201D366
:100510004B00C01A5241411A00D2014652411046C6
:100520007047FFE701B5002000F006F802BDC046A5
:100530000029F7D076E770477047C04630B589B0DC
:100540001422002103A8FFF73FFE134B59698020B6
:10055000C002014359615A6902400192019A5A69E5
:10056000802189020A435A615B690B400293029B16
:100570008025AD01094C00222900200001F038FE41
:1005800003950123049300230593069303A92000F8
:1005900001F062FD09B030BD0010024000040048C7
:1005A00000B583B0094A5169012319435161526969
:1005B00013400193019B00220021092001F000FF5C
:1005C000092001F02FFF03B000BDC046001002401B
:1005D000F0B585B00C22002101A8FFF7F5FD264CEF
:1005E000264B236000236360A360E360012525613F
:1005F0000826666123766376A576E376C222FF320B
:10060000E26123622433E554A562200000F08CFEF1
:1006100080235B01029306270397019501A920001F
:1006200000F0E2FF0223019301A9200000F0DCFFAB
:100630000323019301A9200000F0D6FF04230193B6
:1006400001A9200000F0D0FF0523019301A920009B
:1006500000F0CAFF019701A9200000F0C5FF0723A1
:10066000019301A9200000F0BFFF019601A920001D
:1006700000F0BAFF05B0F0BDA8040020002401403E
:1006800010B598B0302200210CA8FFF79DFD102274
:10069000002107A8FFF798FD1C2200216846FFF7FC
:1006A00093FD30230B932F3B139310930F33119330
:1006B0000BA801F03FF807230793043B089300249D
:1006C00009940A94012107A801F01EFB80239B02D4
:1006D00000930694684601F0B7FB18B010BD000007
:1006E00070B501F085FCFFF7CBFFFFF727FFFFF7A1
:1006F00057FFFFF76DFF02F055FB082240494148C4
:1007000000F0D0FE02F07AFD002815D18026B60157
:100710003D4D01223100280001F06AFDFA246400F9
:10072000200001F087FC00223100280001F060FD6C
:10073000200001F07FFCE9E7344AFE235B00D35C34
:10074000032B06D08021002289012F4801F050FDA3
:10075000F2E78021012289012B4801F049FD12E0D6
:100760008025AD01284C01222900200001F040FD28
:10077000C82001F05FFC00222900200001F038FDB4
:10078000C82001F057FC214AFE235B00D35C032BF9
:10079000E6D18021012289011B4801F029FD02F0E8
:1007A0006BFF00241AE05200194BD0526A00194B1B
:1007B000D15AFFF737FE7F230340174A5355174896
:1007C000C3702300503B4370042102F079FD03F015
:1007D0000FFC022001F02EFC0134E4B2072CD2D829
:1007E00025000F4B1A5D53000549585A084E9B5B74
:1007F0001E003236B042D6DA323B9842ECDCD2E709
:10080000E0010020A804002000040048EC040020BF
:10081000C801002064000020D80100207C000020D6
:100820007400002070B58025AD01094C012229001B
:10083000200001F0DDFC642001F0FCFB0022290017
:10084000200001F0D5FC642001F0F4FBEBE7C0468A
:10085000000400487047FEE77047704710B501F08C
:10086000D7FB10BD10B5024801F055FD10BDC046C4
:10087000F001002010B5024802F016F910BDC04684
:100880003402002082B00A4B996901221143996118
:1008900099690A400092009ADA69802149050A4361
:1008A000DA61DB690B400193019B02B07047C046DF
:1008B0000010024030B589B004001422002103A8C2
:1008C000FFF782FC274B22689A4201D009B030BD65
:1008D000254B996980208000014399619A69024003
:1008E0000092009A596980208002014359615A6937
:1008F00002400192019A5A698021C9020A435A6151
:100900005B690B400293029BFF230393032504952D
:10091000902003A9C00501F09FFB012303930495D8
:100920000025059503A9114801F096FB1048114BCD
:100930000360456085608023C3608033036180234A
:10094000DB0043612023836180235B01C36101F0ED
:100950007FFC002803D1064B23635C62B6E7FFF7F8
:1009600061FFF8E700240140001002400004004845
:10097000F0010020080002404022835A02490B4344
:100980009BB283520020704780BFFFFF4022835AF2
:1009900002490B40835200207047C0467F40000050
:1009A00084B010B503910492059340220123835231
:1009B00000238352043283520C328352FFF7DCFF50
:1009C000002010BC08BC04B018470000F0B50D783A
:1009D000AD0045192B88B14A1340CA78012A54D07A
:1009E000002A48D0022A03D0032A49D0012400E07B
:1009F0000024AB4A13439BB22B800B789E008619D0
:100A000035882DB2A74F3D402B439BB21A4392B27B
:100A100032800B7B002B00D094E04B78002B44D02D
:100A20005023C25A82180B78DB009B188022D20018
:100A300094466344CA88520852001A800B789B007F
:100A4000C3181A88520606D51A883D001540964AE2
:100A50002A4392B21A80CB78012B1BD00B789B00D3
:100A6000C0180388914A134020225A408C4B1343EC
:100A70009BB2038051E08022920013430024B8E728
:100A8000C022D20013430024B3E78022D2001343D4
:100A90000024AEE70B789B00C0180388834A1A40F5
:100AA0007F4B13439BB2038037E05025425B821893
:100AB0000B78DB009B187E4A94466344CA88520830
:100AC00052001A80425B82180B78DB009B18794A2F
:100AD000944663440A69002A21D11A88764D15404C
:100AE000764A2A431A800B789B00C3181A8852044E
:100AF00006D51A886B4D1540714A2A4392B21A8066
:100B00000B789B00C01802886E4B1A40C0239B01D3
:100B10005A40634B13439BB203802000F0BD3E2A32
:100B200006D85508D20700D50135AD021D80DAE799
:100B30005509D20600D1013DAD02ADB25F4A154361
:100B40001D80D0E70B789B00C3181A88554D1540BF
:100B50005D4A2A4392B21A805025425B82180B7874
:100B6000DB009B188022D200944663440A89520815
:100B700052001A80425B82180B78DB009B184C4AAB
:100B8000944663444A89520852001A804B78002BDD
:100B90003AD10B789B00C3181A88520406D51A88DC
:100BA000404D1540464A2A4392B21A800B789B006A
:100BB000C3181A88520606D51A883A4D15403A4A83
:100BC0002A4392B21A800B789B00C3181A88354DBD
:100BD0001540354A2A4392B21A800A789200821848
:100BE0001388384D1D40C0239B016B402C4D2B4377
:100BF0009BB213800B789B00C01803882B4A1340CC
:100C00002B439BB2038088E70B789B00C3181A889C
:100C1000520406D51A88234D1540294A2A4392B218
:100C20001A800B789B00C3181A88520606D51A88BA
:100C30001C4D15401C4A2A4392B21A800B789B0027
:100C4000C3181A88174D15401D4A2A4392B21A80BC
:100C5000CB78012B16D00B789B00C3181A88134D44
:100C60002A40202555400E4A2A4392B21A800B781A
:100C70009B00C3181A8813491140094A0A4392B2CB
:100C80001A804AE70B789B00C3181A88074D154055
:100C9000034A2A4392B21A80E9E7C0468F89FFFFD0
:100CA0008080FFFF8F8FFFFFC080FFFFBF8FFFFFA0
:100CB0000404000006040000FF83FFFF0080FFFF24
:100CC00080C0FFFF8FBFFFFF8081FFFF10B50B7B50
:100CD000002B33D14B78002B18D00B789B00C31816
:100CE0001A88520606D51A884E4C14404E4A2243A2
:100CF00092B21A800B789B00C01803884B4A1A40A6
:100D00004B4B13439BB20380002010BD0B789B001C
:100D1000C3181A88520406D51A88424C1440454A12
:100D2000224392B21A800B789B00C0180388424A73
:100D30001A403F4B13439BB20380E5E74B78002BEF
:100D400037D10B789B00C3181A88520406D51A882D
:100D5000344C1440374A224392B21A800B789B00DD
:100D6000C3181A88520606D51A882E4C14402E4AEB
:100D7000224392B21A800B789B00C3181A88294C20
:100D80001440294A224392B21A800C78A400041914
:100D90002388294A1340264A13439BB223800B78A9
:100DA0009B00C018038821490B401A4392B202806D
:100DB000AAE70B789B00C3181A88520406D51A8834
:100DC000184C14401B4A224392B21A800B789B00A5
:100DD000C3181A88520606D51A88124C1440124AB3
:100DE000224392B21A800B789B00C3181A880D4CCC
:100DF0001440104A224392B21A800C78A4000419BD
:100E000023880A4A13400A4A13439BB223800B7873
:100E10009B00C018038808490B401A4392B2028015
:100E200072E7C0468F8FFFFFC080FFFFBF8FFFFFBD
:100E30008080FFFF80C0FFFF8FBFFFFF4B78002B3C
:100E40000ED10B789B00C01802880C4B1A408023EF
:100E50005B015A400A4B13439BB20380002070474A
:100E60000B789B00C0180388064A134010225A4092
:100E7000034B13439BB20380F0E7C0468FBFFFFFD5
:100E80008080FFFFBF8FFFFF10B50B7B002B39D198
:100E90004B78002B1CD00B789B00C3181A88520685
:100EA00006D51A88184C1440184A224392B21A8068
:100EB000CB78012B26D00B789B00C0180388144AEE
:100EC000134020225A40134B13439BB2038019E076
:100ED0000B789B00C3181A88520406D51A880A4C4E
:100EE00014400D4A224392B21A800B789B00C0181E
:100EF00002880A4B1A40C0239B015A40054B1343FA
:100F00009BB20380002010BD8F8FFFFFC080FFFFCA
:100F1000BF8FFFFF8080FFFF80C0FFFF8FBFFFFFFD
:100F2000002902D14C238022C252002070470000C9
:100F30005822835A02490B439BB2835200207047C8
:100F40000080FFFF4423C05A80B2704700207047E2
:100F500010B501335B0812188020C000844662443B
:100F600007E008784C7824020443148002320231EE
:100F7000013B002BF5D110BD70B505000C00497880
:100F800001292BD0A26923699A4200D8D8E0D21A4D
:100F9000A261227B002A00D0E9E05032A95A6918E8
:100FA0002278D2005218A0498C466244002B00D00F
:100FB000CAE013889D4919409D4B0B431380237849
:100FC0009B00ED182A889B4B1A40C0239B015A4076
:100FD000994B13439BB22B80002070BDA2692369FB
:100FE0009A421DD9D21AA261227B002A1CD02278F3
:100FF000900028180088400664D5002939D1503166
:10100000695A6918D200521887498C466244002BED
:101010001CD111888548084085490143118031E081
:101020000023A3611300DFE79EB2E2883300616909
:101030002800FFF78DFF5023EA5AAA182378DB0017
:101040009B187E4A944663441E802EE03E2B06D8B1
:101050005908D80700D501318902118012E05909D9
:10106000D80600D10139890289B271480143118043
:1010700008E05021695A6918D20052186A498C4612
:101080006244138062899BB261692800FFF760FFA8
:101090006378002B47D123789B00EB181A886849A6
:1010A0001140684A0A4392B21A8023789B00ED18D7
:1010B0002B88654A134030225A405F4B13439BB242
:1010C0002B8089E7002923D15031695A6918D20051
:1010D00052185A498C466244002B06D11188534855
:1010E00008405349014311801BE03E2B06D85908A4
:1010F000D80700D501318902118012E05909D806BC
:1011000000D10139890289B249480143118008E0C0
:101110005021695A6918D200521848498C466244D5
:1011200013802289AFE7012BBFD123789B00EB18F6
:101130001A8843491140454A0A4392B21A80B4E7DB
:101140000023A361130024E73E2B06D85908DB07D0
:1011500000D501318902118031E75909DB0600D140
:101160000139890289B2324B1943118027E70029DE
:1011700010D15022A95A69182278D20052182F494A
:101180008C466244002B1AD111882848084028490F
:10119000014311806278002A37D15032A95A691868
:1011A0002278D200521820498C466244002B19D173
:1011B00013881E4919401E4B0B431380FFE63E2B3C
:1011C00006D85908D80700D5013189021180E1E716
:1011D0005909D80600D10139890289B2144801435E
:1011E0001180D7E73E2B06D85908DB0700D501311F
:1011F00089021180E3E65909DB0600D10139890231
:1012000089B20B4B19431180D9E6012A00D0D6E6EA
:101210004F32A95A69182278D200521802498C46D6
:1012200062441380CBE6C04606040000FF83FFFF44
:101230000080FFFF8FBFFFFF8080FFFF02040000E0
:101240008F8FFFFFC080FFFFBF8FFFFF80C0FFFFBA
:1012500030B55D0812188020C0008446624407E063
:101260001488A4B202320C70240A4C700231013D81
:10127000002DF5D1DB0701D513880B7030BD0000C0
:1012800030B583B0040000230193036899680322FA
:101290000A40012A0ED09968204A114212D19A6858
:1012A00001210A439A601E4B18681E49FFF7BAF8DD
:1012B000019015E01A68D2072DD4DA681204EAD535
:1012C000002008E0A36B10221343A363E36B0F3AE3
:1012D0001343E363012003B030BD019B013B019345
:1012E000019B002BF9D100F09FFE050023681B68CD
:1012F000DB070ED400F098FE401B0228F6D9A36B42
:1013000010221343A363E36B0F3A1343E3630120FB
:10131000E1E70020DFE70020DDE7C046170000809E
:101320008401002040420F0070B5041E00D1B1E0DE
:10133000836B002B7ED0A36BDB0600D5A4E0216875
:101340008B6804221A4000D09EE0A36B52480340F1
:101350000630FF300343A363886803230340012B57
:101360006ED0CB6818208343A0680343CB6021680C
:101370000B699B009B08606803430B612168CB6885
:1013800046480340CB60237E9B03617EC9030B4329
:10139000A17E48030343A06A012858D08020400161
:1013A0000343E06803432069022852D013432422F8
:1013B000A25C52001343E27E012A4CD0E269C221B2
:1013C000FF318A4202D0216A0A4313432168CA6866
:1013D0001A43CA60E26A802149058A420DD0012A77
:1013E0000BD0022A09D0032A07D0042A05D0052AE7
:1013F00003D0062A01D0072A0AD1206841690722B2
:101400009143416120684169E56A2A400A4342618B
:101410002268D26822490A409A422BD0A36B12223A
:101420009343023A1343A363E36B0F3A1343E3631B
:1014300001202EE0C36334228354FFF73BFA7AE79E
:101440000B68DB079AD4CB681B0497D489E710009C
:10145000A6E70422AAE7002903D1802252021343FF
:10146000ACE7A26B20210A43A263E26B1F390A4357
:10147000E263A3E70023E363A36B03229343023AEF
:101480001343A363002004E0A36B10221343A36360
:10149000012070BD0120FCE7FDFEFFFF1902FEFFE9
:1014A000E7FF3F83F8B504000E00170003689B6850
:1014B0005B073ED43423C35C012B3CD03423012290
:1014C000C254437E012B32D0FFF7DAFE051E2CD129
:1014D000A36B1A4A1A4080235B001343A3630023C3
:1014E000E3633422A354236B154A9A62236B154A93
:1014F000DA62236B144A1A6323681C221A6022687A
:10150000536810210B4353602268D3680F390B4393
:10151000D360216840313B003200206B00F0C0FEF8
:101520002268936804210B4393602800F8BD0025CE
:10153000CEE70225F9E70225F7E7C046FEF0FFFFF8
:1015400051150008C3150008CF15000870470000AA
:1015500010B5436A9A6B5021114203D01B6B1B6B71
:10156000984710BD996B802292000A439A631A68CB
:10157000D068C0210901084213D1997E002910D1F9
:10158000116809070DD5916849070ED451680C20E0
:10159000814351609A6B09490A400431FF310A4383
:1015A0009A631800FFF7D2FFDBE79A6B20210A430A
:1015B0009A63DA6B1F390A43DA63F2E7FEFEFFFF34
:1015C000704710B5406AFFF7FBFF10BD704710B5BC
:1015D000406A836B402213438363C36B3C3A1343DB
:1015E000C363FFF7F3FF10BD30B583B004000023E1
:1015F00001933433C35C012B00D18AE034230122F0
:10160000C25403689A68520775D4434A48689042A6
:1016100056D09A6A01200D68A84002439A62E36A94
:101620008022520593421ED0012B1CD0022B1AD0CF
:10163000032B18D0042B16D0052B14D0062B12D058
:10164000072B10D02268506907230340886898420E
:1016500009D05069072398435061206842698D681A
:101660002B40134343610B681A00103A022A4CD8EE
:101670002A4A1268102B0ED0112B09D080235B044C
:101680001343264A13600B68102B07D0002037E065
:101690008023DB03F4E780231B04F1E7204B186869
:1016A0002049FEF7BFFE830018184300019302E0B3
:1016B000019B013B0193019B002BF9D100201FE00E
:1016C0009A6A01200D68A84082439A620B681A004A
:1016D000103A022A1BD8114A1268102B09D0112B7C
:1016E00005D0114B13400D4A1360002008E00F4B4A
:1016F000F8E70F4BF6E7836B202213438363012047
:1017000034230022E25403B030BD0020F8E700206B
:10171000F6E70220F7E7C046011000000827014065
:101720008401002040420F00FFFFFFFEFFFFBFFFCC
:10173000FFFF7FFF70B582B0041E00D185E2036811
:10174000DB072BD5B34B5A680C231340042B1DD059
:10175000B04B5A680C231340082B0ED06368012B42
:1017600041D0002B56D1AB4B1A68AB490A401A60E6
:101770001A68AA490A401A603BE0A64B5B68C0227F
:1017800052021340802252029342E7D1A14B1B68C0
:101790009B0303D56368002B00D159E223689B07A4
:1017A00078D59C4B5B680C221A4262D0994B5A68E0
:1017B0000C231340082B53D0E368002B00D18BE09F
:1017C000944A136801210B43136000F02DFC0500BF
:1017D000904B1B689B0776D400F026FC401B022828
:1017E000F6D9032032E28B4A116880235B020B4357
:1017F00013606368002B25D000F016FC0500854BB4
:101800001B689B03CAD400F00FFC401B6428F6D968
:1018100003201BE2052B09D07E4B1A687E490A4043
:101820001A601A687D490A401A60E2E7794B196824
:101830008022D2020A431A601968802252020A43A7
:101840001A60D6E700F0F0FB0500724B1B689B03A3
:10185000A4D500F0E9FB401B6428F6D90320F5E18C
:101860006C4B5B68C02252021340802212029342EA
:10187000A2D1684B1B689B0704D5E368012B01D0FC
:101880000120E3E163490B68F82293432269D20007
:1018900013430B6023681B0744D5E369002B2ED04C
:1018A0005C4A536A01210B43536200F0BDFB050003
:1018B000584B5B6A9B0735D400F0B6FB401B0228EF
:1018C000F6D90320C2E153490B68F82293432269F9
:1018D000D20013430B60DDE74E4A136801218B43AE
:1018E000136000F0A1FB05004A4B1B689B07D1D594
:1018F00000F09AFB401B0228F6D90320A6E1454AD6
:10190000536A01218B43536200F08EFB0500414B6B
:101910005B6A9B0706D500F087FB401B0228F6D9BF
:10192000032093E123685B0700D47FE0394BDB6938
:10193000DB001DD4374AD169802040050143D161C5
:10194000D36903400193019B0125354B1B68DB05DF
:1019500010D5A368012B21D0002B36D12D4B1A6A4C
:1019600001218A431A621A6A03318A431A621AE011
:101970000025EAE72A4A116880235B000B431360C5
:1019800000F052FB0600264B1B68DB05E1D400F09B
:101990004BFB801B6428F6D9032057E11D4A136ACC
:1019A00001210B431362A368002B24D000F03CFB01
:1019B0000600184B1B6A9B0736D400F035FB801BD2
:1019C000184B9842F5D9032040E1052B09D0114B63
:1019D0001A6A01218A431A621A6A03318A431A6217
:1019E000E1E70C4B1A6A04210A431A621A6A0339A6
:1019F0000A431A62D7E700F017FB0600054B1B6A83
:101A00009B0711D500F010FB801B064B9842F5D9BF
:101A100003201BE100100240FFFFFEFFFFFFFBFF62
:101A20000070004088130000012D3AD02368DB06C7
:101A300010D56369012B3AD0053358D1884A536BCE
:101A400004218B435363536BF4318B43A169C90069
:101A50000B43536323689B0600D482E0804B5A6893
:101A60000C2313400C2B60D07D4B5A680C23134081
:101A7000082B53D0236A002B60D0794A516B802306
:101A80005B020B43536300F0CFFA0500744B5B6BB2
:101A9000DB0366D400F0C8FA401B0228F6D9032005
:101AA000D4E06F4AD3696F490B40D361BEE76C4BFA
:101AB0005A6B04210A435A635A6B03390A435A6327
:101AC00000F0B2FA0500664B5B6B9B0706D400F092
:101AD000ABFA401B0228F6D90320B7E060494B6BF4
:101AE000F8229343A269D20013434B63B2E75C4BE5
:101AF0005A6B04210A435A635A6B03398A435A6367
:101B000000F092FA0500564B5B6B9B07A2D500F0E4
:101B10008BFA401B0228F6D9032097E0504B5B68F4
:101B2000C022520213409342A4D14D4B5B6BDB03A6
:101B300017D5236A012B14D0012087E0484A536B44
:101B400049490B40536300F06FFA0500444B5B6B4F
:101B5000DB0306D500F068FA401B0228F6D9032003
:101B600074E0636A002B00D174E03D4A51680C2296
:101B70000A40082A4DD0022B12D0394A13683B493B
:101B80000B40136000F050FA0400354B1B689B01BA
:101B90003DD500F049FA001B0228F6D9032055E094
:101BA0002F4A136831490B40136000F03DFA0500DD
:101BB0002B4B1B689B0106D500F036FA401B022810
:101BC000F6D9032042E0264BDA6A0F218A43216BC3
:101BD0000A43DA625A6826490A40E16AA06A014368
:101BE0000A435A601968802252040A431A6000F0BE
:101BF0001BFA04001A4B1B689B0106D400F014FA70
:101C0000001B0228F6D9032020E000201EE000205F
:101C10001CE0012B20D0124B5A68D96AC0235B020A
:101C20001340A06A834201D001200FE00F230B4034
:101C3000216B8B4201D0012008E0F0239B031A4066
:101C4000E36A9A420AD0012000E0012002B070BD90
:101C50000120FBE70020F9E70120F7E70020F5E786
:101C600000100240FFFFFFEFFFFFFEFFFFFFFFFE40
:101C7000FF7FC2FF30B589B004AA1F4B180032C8DD
:101C800032C2110002680A606A46103313CB13C2D5
:101C90001B681360194B5A680C231340082B04D09F
:101CA0000C2B26D0164809B030BD910C0F231940DB
:101CB00004A8445C1149C96A0B406946C95CC02349
:101CC0005B021A4080235B029A4208D0C0235B0269
:101CD0009A4209D00A48FEF7A5FB6043E3E70848AB
:101CE000FEF7A0FB6043DEE70648FEF79BFB604380
:101CF000D9E70448D7E7C046B441000800100240C5
:101D000000127A00006CDC0270B504000D0000289F
:101D100000D189E0464B1A68012313408B420BD255
:101D200043490B68012293432B430B600B681A4015
:101D3000AA4201D0012078E023689A070ED55B07FC
:101D400005D53C4A5168E023DB000B435360394A18
:101D50005368F0218B43A1680B4353602368DB0772
:101D600035D56368012B09D0022B24D0032B28D052
:101D7000304A1268920705D4012056E02D4A1268B5
:101D8000920353D52B494A680320824313434B6087
:101D900000F04AF90600274B5B680C221A40636882
:101DA0009B009A4213D000F03FF9801B224B9842CF
:101DB000F1D9032039E01F4A12689201E2D40120D0
:101DC00033E01C4A526BD203DCD401202DE0184BC7
:101DD0001A6801231340AB420BD915490B68012245
:101DE00093432B430B600B681A40AA4201D0012099
:101DF0001BE023685B0706D50E4A53680F490B406A
:101E0000E1680B435360FFF735FF0A4B5A6812092C
:101E10000F2313400A4AD35CD8400A4B18600020B5
:101E200000F0BEF8002000E0012070BD0120FCE7BA
:101E3000002002400010024088130000FFF8FFFF5E
:101E4000004300088401002070B582B004000368DC
:101E5000DB0335D54B4BDB69DB0066D4494AD169DE
:101E6000802040050143D161D36903400193019B68
:101E70000125454B1B68DB0559D5424B1B6AC02227
:101E80009200134013D061680A409A420FD03D4B34
:101E9000186A3E4A02401E6A802149023143196293
:101EA000196A3B4E314019621A62C30753D4354A4E
:101EB000136A36490B4061680B431362012D59D0F8
:101EC0002368DB0706D52F4A136B03218B43A168D8
:101ED0000B43136323689B0706D52A4A136B2D49CE
:101EE0000B40E1680B43136323689B0606D5254A24
:101EF000136B10218B4321690B43136323689B03EE
:101F000006D5204A136B80218B43A1690B431363D1
:101F100023685B0533D51B4A136B40218B436169F2
:101F20000B431363002002B070BD0025A1E7164AE1
:101F3000116880235B000B43136000F075F8060006
:101F4000114B1B68DB0598D400F06EF8801B6428E9
:101F5000F6D90320E7E700F067F80600094B1B6A93
:101F60009B07A4D400F060F8801B0B4B9842F5D976
:101F70000320D8E7D36909490B40D361A0E70020CB
:101F8000D1E7C0460010024000700040FFFCFFFF98
:101F9000FFFFFEFFFFFFFCFF88130000FFFFFFEFC6
:101FA00010B504000F4B1978FA208000FEF73AFABA
:101FB00001000D4B1868FEF735FA00F03FFA0028D3
:101FC0000DD1032C01D901200AE0013000222100AB
:101FD000404200F0F5F9054B1C60002000E00120B4
:101FE00010BDC04680000020840100208400002035
:101FF00010B5064A136810210B4313600020FFF749
:10200000CFFFFEF73FFC002010BDC046002002407D
:10201000034A1168034B1B785B1813607047C04676
:10202000E804002080000020014B18687047C0467B
:10203000E804002070B50400FFF7F6FF0500631CFC
:1020400002D0044B1B78E418FFF7EEFF401BA042C0
:10205000FAD370BD80000020F0B5C64600B582B04E
:10206000002338E0042600E00026AE4035003D4362
:102070000234A400574EA551574C25684246D4431C
:102080002E0026404A68D20302D5424615432E0050
:10209000514D2E606D682E0026404A68920302D58D
:1020A000424615432E004C4D6E60AD682E00264012
:1020B0004A68D20202D5424615432E00464DAE6014
:1020C000ED682C404A68920202D542462A43140029
:1020D000414AD46001330A681400DC4076D00125FF
:1020E0009D402A409046F5D04C68022C01D0122C1D
:1020F0000ED1DC080834A400275807261E40B6007D
:102100000F22B24097430A69B24016003E43265060
:1021100002685F0003242600BE40F6433240944626
:102120004A681440BC406246144304604C68621E16
:10213000012A03D9112C01D0122C10D1846834400B
:10214000A446CC68BC406246144384604468AC43F7
:102150004A681209012515409D4025434560C46821
:1021600026408C68BC403443C4604A68D200B1D574
:102170001A4DAE6901242643AE61AD692C4001942D
:10218000019C9C08A51CAD00124EAF5903261E40B1
:10219000B5000F26AE40B7439026F605B04200D1F9
:1021A00062E70F4EB0420BD00E4EB0420AD00E4E38
:1021B000B04209D00D4EB04200D153E7052654E796
:1021C000012652E7022650E703264EE702B004BC80
:1021D0009046F0BD000001400004014000100240A4
:1021E0000004004800080048000C004800100048A7
:1021F000002A01D1816270478161FCE770B5C56B2F
:102200000124066CB4406C60046863604368102B62
:1022100004D0036899600368DA6070BD03689A604F
:102220000368D960F9E7000010B504000368064AA6
:102230009446634418001421FEF7F4F880002064EB
:10224000024BE36310BDC046F8FFFDBF0000024033
:1022500070B5041E20D021250223435501680B6868
:102260000E4A1A40436880680343E06803432069CC
:10227000034360690343A0690343E06903431343D5
:102280000B602000FFF7D0FF0023A36301226255FB
:102290001F32A354002070BD0120FCE70FC0FFFFD8
:1022A00070B504002020205C012832D020200125B8
:1022B00025540130205C012804D020230022E25460
:1022C000022070BD2030013525540020A063256810
:1022D00028680126B04328602000FFF78FFFE36ADB
:1022E000002B0BD0226813680E210B431360226869
:1022F000136801210B4313600020E2E72268136892
:102300000A210B4313602268136806398B4313605C
:10231000EDE70220D5E770B5C36B1A68046825683D
:10232000016C04238B401A4212D06B0710D523682E
:102330009B0603D42368042293432360C26B0423C7
:10234000016C8B405360C36A002B00D0984770BD6E
:1023500002238B401A4218D0AB0716D523689B0680
:1023600006D423680A22934323602123093AC254E6
:10237000C26B0223016C8B40536020230022C254A5
:10238000836A002BE3D09847E1E708238B401A4289
:10239000DDD02B07DBD523680E2293432360C26B6D
:1023A00001231900046CA1405160836321228354EE
:1023B0001F330022C254036B002BC8D09847C6E7D6
:1023C00070B5002811DB8308144DC0339B005C59A5
:1023D00003221040C000FC3216008640B44389013D
:1023E0000A40824022435A5170BDC0B20F230340BD
:1023F000083B9B0806339B00094A944663445D688A
:1024000003242040C000FF2214008440A54389011A
:102410001140814029435960E6E7C04600E100E0F1
:1024200000ED00E0002805DB1F2318401E3B834021
:10243000014A13607047C04600E100E001380A4BD2
:1024400098420FD8094A50600948036A1B021B0AC8
:10245000C02109060B430362002393600733136016
:10246000002070470120FCE7FFFFFF0010E000E0C4
:1024700000ED00E030B587B0041E61D0314BC35C85
:10248000002B07D02F4B0322E2542068FEF77EFA80
:1024900000231AE08A239B000022C25400F09EFC15
:1024A000F0E75A01A2181100293101200870013902
:1024B0000B70D38610002B30002101709163D16323
:1024C0009A1C520111510133DBB260688342E8D398
:1024D000002215E05301E3181D002A35FF350021C5
:1024E0002970013D2A70033529700D3529603D336F
:1024F000FF33196013000A335B0119510132D2B264
:102500009042E7D86A462300103323CB23C203CB83
:1025100003C26168A268E3682068FEF741FA2423D9
:102520000022E254074B0132E254E369012B02D04E
:10253000002007B030BD200000F01FFC0020F8E7AD
:102540000120F6E72902000070B504008A239B00F1
:10255000C35C012B0DD08A25AD00012343550068D3
:10256000FEF7E6FC2068FEF707FA0023635500201B
:1025700070BD0220FCE770B504008A239B00C35C99
:10258000012B0CD08A25AD00012343552333C154C0
:102590000068FEF7C5FC00236355002070BD0220D3
:1025A000FCE770B5050048B2002827DB07240C4083
:1025B000640120002930FF3028182C192A34FF34F8
:1025C000002626700724214001700261C370427802
:1025D000002A00D0C181022B1BD08A239B00EB5C18
:1025E000012B19D08A24A40001232B55010028684F
:1025F000FEF7ECF900232B55002070BD07240C409A
:1026000064012000283028182C192934012626704E
:10261000D8E700230371E0E70220EEE770B504007D
:102620004BB2002B1FDB07230B405B011A00293242
:10263000FF328218C3182A33FF3300201870072393
:10264000194011708A239B00E35C012B16D08A2568
:10265000AD000123635511002068FEF737FB00230E
:102660006355002070BD07230B405B011A00283220
:102670008218C318293301201870E0E70220F1E71F
:1026800070B507250D406C0121002931FF3141183B
:10269000041926003D36FF3632602A000A32520104
:1026A000135082180023536022002A32FF32137025
:1026B0002934FF342570002D04D00068FEF75CFC3F
:1026C000002070BD0068FEF757FCF9E770B50725DC
:1026D0000D406C012100283141180419E263AA1C45
:1026E0005201135082180023536023002933012222
:1026F0001A7028342570002D04D00068FEF73CFCC9
:10270000002070BD0068FEF737FCF9E7F0B5C6465B
:1027100000B5050028684423C35A1BB2002B00DB18
:10272000AAE14423C35A9BB20F241C4000D0BCE052
:10273000DB0651D503889BB21A0500D57FE01BB29A
:10274000002BE7DA0388CE4A13408022134303802C
:1027500028685023C35A94225200AA5CD2009B18C6
:102760001B18C84A944663441B889B059B0D2A008E
:102770002932FF32D361002B0FD0516900290CD0D0
:102780001400D288FEF764FD6369E26994466344ED
:1027900063610021280000F04CFB2B6850229A5AFC
:1027A0009B18B84A944663442A002932FF321269C2
:1027B000002A67D11A88B4491140B44A0A431A80E2
:1027C00029680A88B24B1A40C0239B015A40B14B7A
:1027D00013439BB20B809DE70388AF4A1A40AB4B73
:1027E00013439BB2038029685023CB5A2822AA5C4A
:1027F000D2009B185B18A94A944663441B889B052A
:102800009B0D6B64EA6B94466344EB6300212800E4
:1028100000F01CFB2423EB5C002B00D17AE72B6C2F
:10282000002B00D076E72422AB5C802149420B4389
:10283000DBB2CC31286843520023AB546AE7502303
:10284000C35A94225200AA5CD2009B181B188D4ACE
:10285000944663441B889B059B0D2A002932FF3256
:10286000D3618C2189006918D288FEF7F1FC2A68AF
:10287000138883490B4080210B431380280000F00C
:10288000CDFA47E73E2A06D85108D20700D50131D4
:102890008902198094E75109D20600D101398902D1
:1028A00089B27A4A114319808AE7A30098464044C6
:1028B0000688B6B233B2002B30DB330600D429E7EA
:1028C0002B6843441A001B88734919406F4B0B4314
:1028D0009BB2138028685023C35A610169180A000B
:1028E00028321278D2009B181B186C4A9446634415
:1028F0001A889205920DA31C5B01E8184260C86B10
:1029000084466244CA635B59002B00D0ACE00C00E3
:1029100028342178280000F099FAFBE60388584A09
:1029200013408022134303806301EB183533FF33D8
:102930001B78002B1ED128685033C35A6201AA1895
:102940002932FF321278D2009B181B184D4A944648
:1029500063441F88BF05BF0D33D06301EB181A0015
:102960002F32FF3212883D33FF3319683B00FEF7E8
:102970006FFC26E028686301EB182933FF331B78CE
:102980009A008218128852044BD55022825ADB00DA
:10299000D3181B18414A944663441F88BF05BF0DD6
:1029A00032D16301EB182933FF331A7892002B6878
:1029B0009C46624413883A4919403A4B0B439BB2F8
:1029C0001380390020000A3040012A185368DB19AF
:1029D00053606301EB183D33FF331A689446674434
:1029E0001F604359002B06D06201AA183932FF320A
:1029F000126891422ED26301EB182933FF33197804
:102A0000280000F016FA58E76301EB181A0031327B
:102A1000FF3212883D33FF3319683B00FEF718FC84
:102A2000BFE75022825ADB00D3181B18154A944680
:102A300063441F88BF05BF0DB3D06301EB181A00B4
:102A40003332FF3212883D33FF3319683B00FEF703
:102A5000FFFBA6E76201AA182932FF3211783A007B
:102A60002800FFF70DFE28E764012C19283421788F
:102A70002800FFF72BFE4DE6002004BC9046F0BD79
:102A80008F0F000006040000FF83FFFF0080FFFFA0
:102A90008FBFFFFF8080FFFF0F8FFFFF020400004A
:102AA0008F8FFFFFC080FFFF70B504000068FEF746
:102AB00049FA030400D57BE02068FEF743FA43059A
:102AC00000D579E02068FEF73DFA430405D521687A
:102AD00044228B5A584803408B522068FEF732FA42
:102AE000830405D5216844228B5A544803408B52F5
:102AF0002068FEF727FAC30418D521684023CA5A74
:102B000004208243CA522168CA5A04308243CA52FE
:102B100098239B00E35C012B5CD0200000F0C6F9F9
:102B2000216844228B5A464803408B522068FEF7A6
:102B300009FA030557D42068FEF704FA030626D5E0
:102B4000216844228B5A802083438B5298239B0018
:102B5000E35C002B62D121684033CA5A042002434F
:102B6000CA522168CA5A08200243CA5298239B00BD
:102B70000122E25454232268D25A9208183B13408F
:102B800099229200A3500121200000F009F9206849
:102B9000FEF7D8F9830545D42068FEF7D3F9C305BD
:102BA00005D5216844228B5A264803408B5270BDBC
:102BB0002000FFF7ABFD7FE7216844228B5A2248B3
:102BC00003408B52200000F053F900212000FFF752
:102BD000D2FC77E798239B000022E25400212000DA
:102BE00000F0DEF899E721684023CA5A0820024322
:102BF000CA5220684421425A144D2A404252216848
:102C0000CA5A04200243CA522068FEF79BF9C30443
:102C100000D590E7200000F037F98CE7200000F0A5
:102C200033F9B4E7216844228B5A094803408B5298
:102C3000200000F016F9AFE7FFBFFFFFFFDFFFFF47
:102C4000FFEFFFFFFFFEFFFFFFFBFFFFFFF7FFFFB1
:102C5000FFFDFFFF70B5050007240C4043689C4250
:102C600033D84BB2002B20DB4B0119002931FF3147
:102C70004118C3182A33FF3300221A7001238B70C6
:102C80000C708A239B00EB5C012B20D08A239B00D5
:102C90000122EA542868FEF7D1F8002C0ED08A23CE
:102CA0009B000022EA54002010E063011900283143
:102CB0004118C318293301221A70DFE78C239B00C7
:102CC000E9182868FEF742F9E9E7012070BD022003
:102CD000FCE770B504000F230B40426893422FD8E5
:102CE0004BB2002B21DB07230B405B011A0029327A
:102CF000FF328218C3182A33FF33002018700023D4
:102D000093700733194011708A239B00E35C012BF9
:102D100018D08A25AD000123635511002068FEF705
:102D2000B3F80023635500200BE007230B405B0141
:102D30001A0028328218C318293301201870DEE7E0
:102D4000012070BD0220FCE710B50C060DD507244C
:102D50002140490128314018002A0BD0012202737A
:102D600003811B0C4381002010BD49012931FF3133
:102D70004018F1E70273C380F5E702689A239B00CD
:102D80000121C150083B0021C1545423D15A0120D4
:102D90000143D152D15A02200143D1520020704741
:102DA0007047000010B5094C00220949200000F0CE
:102DB00079FC0849200000F091FC0749200001F04F
:102DC00067F9200000F093FC10BDC046EC04002021
:102DD00088000020C4000020BC00002000B583B0A3
:102DE00002680C4B9A4201D003B000BD0A4AD16977
:102DF000802000040143D161D36903400193019B0A
:102E0000002201211F20FFF7DBFA1F20FFF70AFB3A
:102E1000EAE7C046005C00400010024010B5010027
:102E20009C239B00C058403B9C46614400F07CFCC6
:102E300010BD10B503009C22920080584A019B18D7
:102E40003D33FF331A6800F0A3FC10BD10B503003A
:102E50009C22920080584A019B18DA6B00F0D4FC47
:102E600010BD10B59C239B00C05800F066FD10BD3E
:102E700070B505009C24A4000121005900F048FD14
:102E8000285900F022FD70BD10B504009C239B0062
:102E9000C05800F040FDA369002B04D0024A13691A
:102EA00006210B43136110BD00ED00E010B59C231B
:102EB0009B00C05800F03AFD10BD000070B5040042
:102EC0001B489C239B00C4508825AD006051194BC2
:102ED000036008234360022282600023C360026112
:102EE0008361C3610362FFF7C5FA18230022002142
:102EF0006059FFF729FF5823002280216059FFF70E
:102F000023FFC023002281216059FFF71DFF882382
:102F10005B00002201216059FFF716FF60598023F2
:102F20005B0000228221FFF70FFF002070BDC0462A
:102F300034020020005C004010B588239B00C0587C
:102F4000FFF702FB002803D0022803D0022010BDA7
:102F50000020FCE70120FAE710B514001A008823CE
:102F60009B00C0582300FFF71CFB002803D0022859
:102F700003D0022010BD0020FCE70120FAE710B5C5
:102F800088239B00C058FFF749FB002803D0022884
:102F900003D0022010BD0020FCE70120FAE710B5A5
:102FA00088239B00C058FFF755FE002803D0022855
:102FB00003D0022010BD0020FCE70120FAE710B585
:102FC00088239B00C058FFF784FE002803D0022806
:102FD00003D0022010BD0020FCE70120FAE70A0020
:102FE00088239B00C35849B2002907DB7F21114089
:102FF00049015B182B33FF33187870477F2111404C
:1030000049015B182A331878F7E710B588239B002D
:10301000C058FFF7B0FA002803D0022803D00220DE
:1030200010BD0020FCE70120FAE710B58824A400B9
:103030000059FFF74BFB002803D0022803D00220E1
:1030400010BD0020FCE70120FAE710B58824A40099
:103050000059FFF715FB002803D0022803D00220F7
:1030600010BD0020FCE70120FAE7000012230B80CE
:1030700000487047A400002004230B8000487047DC
:10308000B800002010B50A00002805D00549064800
:1030900000F001FF034810BD0249034800F0FBFEA9
:1030A000F8E7C046100700200442000810B50A00E7
:1030B000034C2100034800F0EEFE200010BDC04686
:1030C00010070020F041000810B50A00002805D0C4
:1030D0000549064800F0DFFE034810BD02490348D9
:1030E00000F0D9FEF8E7C0461007002010420008A3
:1030F00010B50A00002805D00549064800F0CBFEAF
:10310000034810BD0249034800F0C5FEF8E7C04679
:1031100010070020D441000810B50A00002805D08F
:103120000549064800F0B7FE034810BD02490348B0
:1031300000F0B1FEF8E7C04610070020E0410008AB
:1031400070B5002291420FD9084C2368865C084D67
:10315000EE5401332360013280246400A342F1D194
:10316000024B00241C60EDE7002070BDB801002078
:10317000B4090020F0B5DE46474680B585B00600AC
:103180008B089B4603270F40019727D0002005B0EE
:103190000CBC90469B46F0BD00230093019C18E0B8
:1031A00002230093FAE703230093F7E70123009338
:1031B000F4E74346E3180133F35C02AAD11D0B7018
:1031C0006B005B1998000B4BC01800F091FF0134A5
:1031D000A4B26B461B88A342EBD80137BB45D5D9B7
:1031E000BB009846F25C15090F2313409B00024A6E
:1031F000D3589F46640900202042000810B50024DF
:10320000002C07D00024002C11D0002000281BD057
:10321000012010BD802163001B199800194BC018B4
:10322000890000F04BFF012827D10134E8E7802115
:1032300063001B199800144BC018890000F03EFF72
:1032400001281CD10134DEE70022104B1A54810002
:103250000F4B5B18DA7083011B180E495A54020099
:1032600007E0810109180B4B5B189B18002159706E
:1032700001323F2AF5D90130C8E70020C9E7002014
:10328000C7E7C04664090020100900201C0900207F
:10329000700900202009002010B50749411843009B
:1032A000181883000548181800F03AFF012801D0CB
:1032B000002010BD0120FCE71C090020100900209F
:1032C00010B5042900D010BDFFF73AFFFBE700005E
:1032D000F0B58F4B1A5C0F23110099430B0049B2D4
:1032E000002924DB83008B495B5C022B00D1DCE0EE
:1032F00000D8B7E0032B00D1EEE0042B60D18101B0
:103300000918854B5B189A708200824B9B185B787A
:10331000042B00D1F5E0032B52D183011B187E4A08
:103320000221995483007B4A0231995448E0B02B22
:1033300000D188E010D9D02B21D01ED9E02B00D1AC
:1033400081E0F02B11D113001033D9B20F2932D8FC
:103350008B007249CB589F46902B00D173E0A02B75
:1033600000D170E0802B00D16DE06A4984000A1919
:10337000002353706354937022E0C02BF5D1810178
:103380000918654B5B185A70624A81005318032470
:103390005C70023C8C5400229A7011E05D4C8500F8
:1033A00066190127F770810109185B4B5B185A7089
:1033B000777003232B558200564B9B1801229A707D
:1033C0008000544BC35C042B00D19FE00020F0BD73
:1033D000504D8600AB19D9788C460131C9B2D970ED
:1033E0004D4F83011B18FC1864446270D9550423A7
:1033F0007355E0E781010918474B5B185A70454B3C
:103400008200991804244C700121D154D3E7810122
:103410000918414B5B185A703E4B820099180324DF
:103420004C700121D154C6E73B4983011B18CC18CD
:10343000627001225A54374B8200991802244C7052
:103440000421D154B7E781010918334B5B185A7036
:10345000304A8100531804245C70033C8C540022D1
:103460009A70ADE7012BABD1810109182A4B5B188B
:103470009A708200274B9B185B78042B06D0032B95
:1034800009D08300234A0021995499E71300214A67
:103490000221995494E783011B181F4A0221995471
:1034A00083001C4A023199548AE78100194B5B184A
:1034B0005B78042B04D08300164A002199547FE7DF
:1034C000154983011B18CC18E27003225A5483005B
:1034D000104A0421995473E783000E4CE418E578F0
:1034E000691CC9B2E170840124180B4B1B195B19CC
:1034F0005A703F2900D863E78300064A0421995493
:103500005EE71300034A0221995459E701205EE760
:103510001C090020700900202009002060420008DA
:10352000F0B583B007000023019304008200504BE4
:103530009B185B78022B18D004D8012B23D10026CE
:1035400000257CE0042B1ED88200494B9B189B78F9
:10355000002B1CD00301DBB282011718454ABA5C6C
:103560009B1801AA1370002127E00301DBB282013E
:103570001218404FBF187A7812099B1801A80370DF
:103580000421FFF79DFE00F033FD03B0F0BD030101
:10359000DBB282011218374FBF187A7812099B18D4
:1035A00001AA1370DFE7481CA2011219314B9B18C6
:1035B0005B185A7801AB1A540100A20112192D4B65
:1035C000D35C8B42EFD8042101A8FFF779FEDAE73C
:1035D00001A8C3703B01DBB2043303700421FFF781
:1035E0006FFE3FE0012D1CD0002D0CD0022D39D1F3
:1035F0003B01DBB2073301A80370F723C37004213A
:10360000FFF75EFE2EE03B01DBB2053301A803703D
:10361000F72343700023C37083700421FFF750FE2B
:1036200020E03B01DBB2063301A80370F72383706F
:103630000023C3700421FFF743FE13E00136A3010A
:103640001B190C4A9B5CB3429DD9A2011219094B6C
:103650009B189B195B78F72BC4D0022DB8D06A1C3D
:1036600001A98B540135022DE8D90025E6E7C046B3
:10367000700900202009002070B50025002D00D021
:1036800070BDECB22000FFF707FE012808D1200032
:10369000FFF71EFE0028F4D02000FFF741FFF0E7FF
:1036A0000135EBE710B5002816D085239B00C358E1
:1036B000002B03D085239B000024C450002902D096
:1036C00084239B00C150FE235B000121C154027082
:1036D000FFF7F4FB002010BD0220FCE7002904D016
:1036E00085239B00C150002070470220FCE710B5E5
:1036F000FFF722FC002010BD10B585239B00C358A6
:10370000002B07D01B689847002801D1002010BD6E
:103710000220FCE70220FAE710B585239B00C3587E
:103720005B689847002010BD70B5040082239B00A1
:10373000C518280000F02CF9FA235B000122E250A2
:10374000124BE25A163BE2501033E15CEA3BFF3B7E
:103750000B40012B0FD0002B07D0022B10D07F2362
:1037600099432000FFF71BFC03E02900200000F034
:10377000B3FA002070BD2900200000F0D1FAF8E76C
:103780002900200000F0EBFAF3E7C0460E0200002B
:1037900010B504001300002929D1FA2252008258E2
:1037A000032A01D0002010BD421DFF329168D2686B
:1037B00091420FD885239B00C3581B69002B05D06D
:1037C000FE225200825C032A00D19847200000F0BC
:1037D0009EFBE7E7891A0530FF3081608A4200D9F5
:1037E0000A0092B21900200000F089FBDAE7852375
:1037F0009B00C3589B69002BD4D0FE225200825CF0
:10380000032ACFD19847CDE770B5040013000029F3
:103810004ED1FA2252008258022A06D080239B0001
:10382000E35C012B3FD0002070BDC269056AAA424B
:103830001ED8866929003000FCF77AFE002906D1DF
:10384000B54204D8FC235B00E3589E421DD3852378
:103850009B00E358DB68002B06D0FE225200A25CDE
:10386000032A01D120009847200000F05CFBD5E737
:10387000521BC26192B2190000F039FB00230022F2
:1038800000212000FFF7E1FBC8E70022200000F044
:103890002EFBFC235B000022E250002300212000CD
:1038A000FFF7D3FBBAE780239B000022E254BAE77C
:1038B00085239B00C3585B69002BB4D0FE225200C5
:1038C000825C032AAFD19847ADE770B5040040236E
:1038D00000220021FFF740FB402588235B00E550D4
:1038E000D03B002280212000FFF736FB2562FE231B
:1038F0005B000122E2541C33E358002B06D08523E1
:103900009B00E3585B68217920009847002070BD38
:10391000017400207047FE235B00C15CFE22FF3271
:103920008154FA3AFF3AC25400207047FE23FF3315
:10393000C25C013BC2540020704710B5FE235B00FF
:10394000C35C032B01D0002010BD85239B00C3580E
:10395000DB69002BF7D09847F5E70300002002E071
:103960000130C0B201331A78002AF9D1704710B57E
:1039700004004B88012B0AD181239B000122C250F5
:103980001033C3589B689847200000F0C0FA10BD60
:103990000B7803704B7843708B78CA7812029B18AF
:1039A00043800B794A7912029B1883808B79CA79FC
:1039B00012029B18C380704710B504008021FFF7E6
:1039C000EEFA00212000FFF7EAFA10BD30B583B00F
:1039D00004000D004A88130A072B00D98EE09B00D3
:1039E0004F49CB589F4684239B00C3581B68007CDB
:1039F0006A46911D98476B4606331B88002B03D0FF
:103A0000EA88002A00D07EE003B030BD037C002BA2
:103A100009D185239B00C3589B6A6A46901D98472D
:103A200002234370E7E785239B00C358DB6A6A469D
:103A3000901D984702234370DDE7D2B2052A39D89A
:103A40009200384B9B589F4684239B00C3585B6869
:103A5000007C6A46911D9847CDE784239B00C3589C
:103A60009B68007C6A46911D9847C4E784239B00AD
:103A7000C358DB68007C6A46911D9847BBE78423E6
:103A80009B00C3581B69007C6A46911D9847B2E7AA
:103A900084239B00C3585B69007C6A46911D98474C
:103AA000A9E784239B00C3589B69007C6A46911D4B
:103AB0009847A0E72900FFF77FFFA5E7037C002BCD
:103AC00007D185239B00C3585B6B6A46901D9847BE
:103AD00091E72900FFF770FF96E7037C002B09D1DF
:103AE00085239B00C3581B6B6A46901D984707238C
:103AF000437080E72900FFF75FFF85E7290020007A
:103B0000FFF75AFF80E7191C934200D9111C8AB2B3
:103B10006B46D9800100200000F0DBF974E7C04655
:103B2000A0420008C042000870B504008B88002B3A
:103B300022D1CB88002B1FD18B787F251D40FE23FF
:103B40005B00C35C032B0FD0FF235B00C55429002F
:103B5000FFF75BFA200000F0DAF9002D07D0FE2312
:103B60005B000222E2540AE0FFF726FF07E0FE2393
:103B70005B000122E25402E02000FFF71DFF70BD50
:103B800070B504000D008978284B197001290AD8F6
:103B9000FE235B00C35C022B09D0032B1ED029003F
:103BA000FFF70AFF02E02900FFF706FF70BD0029BA
:103BB00011D04160FE235B000322C254FFF79CFD3D
:103BC000022803D0200000F0A2F9EFE7290020002E
:103BD000FFF7F2FEEAE700F09AF9E7E7002911D0D3
:103BE000436899421ED0D9B2FFF796FD0F4B197862
:103BF00061602000FFF780FD02280ED0200000F059
:103C000086F9D3E7FE235B000222C2544160FFF72E
:103C100083FD200000F07BF9C8E729002000FFF7B2
:103C2000CBFEC3E700F073F9C0E7C046B001002047
:103C300010B5CB88012B09D1FE235B00C35C022B9E
:103C400007D0032B0DD0FFF7B7FE01E0FFF7B4FE5E
:103C500010BD0023836001000831012200F039F912
:103C6000F6E7011D012200F034F9F1E710B5FE235B
:103C70005B00C35C023BDBB2012B0ED80123C360A7
:103C800081239B00C358002B01D00323C360010094
:103C90000C31022200F01DF910BDFFF78DFEFBE78D
:103CA00010B50400FE235B00C35C023BDBB2012BBA
:103CB0000ED84B88012B0AD181239B000022C250D1
:103CC0001033C3589B689847200000F020F910BDBE
:103CD000FFF772FEFBE7000010B54B78092B19D8EF
:103CE0009B000E4AD3589F46FFF770FE002010BD80
:103CF000FFF71AFFFAE7FFF743FFF7E7FFF798FF31
:103D0000F4E7FFF7B3FFF1E7FFF731FEEEE7FFF768
:103D1000C7FFEBE7FFF750FEE8E7C046D8420008D0
:103D200070B504000D00FE235B00C35C032B13D1B0
:103D30000B79012B0DD885239B00C3589B689847AE
:103D4000EB88002B01D0002070BD200000F0DFF8D0
:103D5000F9E7FFF731FEF6E7FFF72EFEF3E770B560
:103D600005000C008A88D1B2207860230340202B04
:103D700008D1F533FF33EB589B68210028009847A2
:103D8000002070BD6378012B2CD0002B52D0032B68
:103D9000F6D1FA33FF33EB5C022B06D0032B0CD0A9
:103DA00021002800FFF708FEEAE70029E8D0802973
:103DB000E6D02800FFF7F3F8E2E76388002B06D18E
:103DC000002904D0802902D02800FFF7E8F88523D5
:103DD0009B00EB589B68210028009847280000F0C2
:103DE00096F8CDE7FE235B00EB5C022B06D0032B9D
:103DF0000CD021002800FFF7DFFDC1E70029BFD06C
:103E00008029BDD02800FFF7CAF8B9E76388002BE6
:103E1000B6D14B0603D1280000F079F8B0E72800AE
:103E2000FFF7CDF885239B00EB589B682100280005
:103E30009847F0E7FE235B00EB5C022B06D0032BD8
:103E40000AD021002800FFF7B7FD99E74B0697D06D
:103E50002800FFF7A4F893E7130612D47F240C4040
:103E6000103424012C1904342800FFF7B8F8002876
:103E70000ED00123236002222100280000F029F83F
:103E80007EE77F240C40013424012C190434EBE735
:103E900000232360EFE770B504000D001600002832
:103EA00016D0FFF75AFD0130400080B230802870F4
:103EB00003236B70013B08E001345A1CD2B2E95471
:103EC0000233DBB2AA180021117021780029F3D146
:103ED00070BD10B51300FA22520002248450836191
:103EE000C3610A000021FFF7A0F8002010BD10B543
:103EF00013000A000021FFF798F8002010BD10B54C
:103F000013000A000021FFF7A0F8002010BD10B533
:103F1000FA235B000422C250002300220021FFF795
:103F200084F8002010BD10B5FA235B000522C250B2
:103F3000002300220021FFF788F8002010BD0000B8
:103F4000044B1B78012B01D000207047014B00224D
:103F50001A70F9E7C00100208523038000487047EC
:103F6000FC00002070B5040087239B00C258043376
:103F7000C3580A314901591889881368054D28002A
:103F8000984740232A0001212000FFF75EF8002017
:103F900070BDC0467409002010B50400054B002216
:103FA0001A608121FEF7EBFF01212000FEF7E7FFF9
:103FB000002010BDC401002010B504000A4B186099
:103FC000402302228121FEF7C7FF40230222012164
:103FD0002000FEF7C1FF4023044A01212000FFF723
:103FE00034F8002010BDC046C40100207409002030
:103FF00010B5214B1B78012B28D0204B1A68802349
:104000005B009A4223D01D4B19681D4B1B689942D7
:1040100021D024D980235B005B1A1A4A1360194B04
:10402000186840281FD98AB20B00403313490B602F
:104030004038144B186040230F4901200870124982
:104040005218124908688121FEF7EFFF10BD0B4B93
:1040500000221A60D7E7084B00221A70F6E75B1AB5
:10406000084A1360DBE78AB283B20918034801608B
:10407000044900200860DFE7C0010020BC010020E7
:10408000B8010020B4010020B4090020C4010020C0
:10409000002904D087239B00C150002070470220D4
:1040A000FCE710B504008068002801D0FCF782F816
:1040B000002363802380A380012010BD70B505001C
:1040C0000C00FFF7EEFF26002000FCF769F8A8605F
:1040D00000280BD0002304E0AA68D2180021117038
:1040E00001339E42F8D8AC80012070BD0020FCE76F
:1040F00010B50288541C8388013B23404488A342A6
:104100000CD00B7881688B54038801339BB2828872
:10411000013A12B213400380012010BD0020FCE7D9
:10412000028843889A420CD08268D35C0B70438823
:1041300001339BB28288013A12B2134043800120BE
:1041400070470020FCE770470D4885460D480E4932
:104150000E4A002302E0D458C4500433C4188C42E1
:10416000F9D30B4A0B4C002301E013600432A24246
:10417000FBD3FFF7E8FFFBF7EFFFFCF7B1FAFEE731
:1041800000400020000000208801002018430008A3
:1041900088010020B80A0020FEE70000F8B5C046FC
:1041A000F8BC08BC9E467047F8B5C046F8BC08BCD1
:0441B0009E46704770
:1041B40002030405060708090A0B0C0D0E0F101064
:1041C4000102030405060708090A0B0C0D0E0F1063
:1041D4004D49444920436F6E666967004D4944491F
:1041E40020496E7465726661636500004F7474657E
:1041F4007220536369656E74696669630000000028
:104204004D494449204469616C73000030303030BA
:104214003030303030303141000000009831000837
:1042240098310008A0310008A6310008A631000822
:10423400AC310008A0310008A6310008A6310008FE
:10424400A6310008A6310008A6310008A0310008F4
:10425400A0310008A6310008AC3100089C330008E6
:104264000E340008F43300080E3400082834000823
:104274002834000828340008D03300082834000803
:10428400283400082834000828340008283400089A
:10429400283400082834000828340008FC3A0008B0
:1042A400E63900080C3A00083A3A0008FC3A0008DB
:1042B400FC3A0008BC3A0008DA3A0008483A000818
:1042C4005A3A00086C3A00087E3A0008903A00080E
:1042D400A23A0008023D00080E3D0008143D000803
:1042E400083D0008143D0008F03C0008E83C0008C4
:1042F400143D0008FC3C0008F63C000800000000E7
:0C43040000000000010203040607080985
:04431000350100086B
:044314000901000893
:104318000400002000000000000000000000000071
:104328000000000000000000000000000000000085
:104338000000000000000000000000000000000075
:104348000000000000000000000000000000000065
:104358000000000000000000000000000000000055
:104368000000000000000000000000000000000045
:104378000000000020002000200020002000200075
:104388002000000101020304050607000BB000002D
:1043980001000000040000006D30000879300008BA
:1043A800AD30000885300008C9300008F130000839
:1043B800193100081201000202020040091201002E
:1043C8000002010203010000040311047531000812
:1043D80041310008B93F0008993F0008000000007B
:1043E8000000000000000000413F0008653F000891
:1043F80000000000000000000000000000000000B5
:10440800593F000800000000000000000902850074
:10441800020100800A0904000000010100000924CB
:104428000100010900010109040100020103000063
:1044380007240100014300062402010100062402AA
:1044480002020006240201110006240202120009D9
:1044580024030103010201000924030204010101EC
:1044680000092403011301120100092403021401A5
:1044780011010009050102400000000006250102A3
:104488000111090581024000000000062501020310
:084498001300000000127A007D
:040000050800414965
:00000001FF
